BL51 BANKED LINKER/LOCATER V6.00                                                        07/23/2018  09:53:49  PAGE 1


BL51 BANKED LINKER/LOCATER V6.00, INVOKED BY:
C:\KEIL\C51\BIN\BL51.EXE main.obj, Delay_1T.obj TO MA82G5Dxx RAMSIZE (256)


MEMORY MODEL: SMALL


INPUT MODULES INCLUDED:
  main.obj (MAIN)
  Delay_1T.obj (DELAY_1T)
  C:\KEIL\C51\LIB\C51S.LIB (?C_STARTUP)


LINK MAP OF MODULE:  MA82G5Dxx (MAIN)


            TYPE    BASE      LENGTH    RELOCATION   SEGMENT NAME
            -----------------------------------------------------

            * * * * * * *   D A T A   M E M O R Y   * * * * * * *
            REG     0000H     0008H     ABSOLUTE     "REG BANK 0"
            DATA    0008H     0001H     UNIT         ?DT?MAIN
            IDATA   0009H     0001H     UNIT         ?STACK

            * * * * * * *   C O D E   M E M O R Y   * * * * * * *
            CODE    0000H     0003H     ABSOLUTE     
            CODE    0003H     001DH     UNIT         ?PR?INT_UART0?MAIN
                    0020H     0003H                  *** GAP ***
            CODE    0023H     0003H     ABSOLUTE     
            CODE    0026H     00A9H     UNIT         CODE_DELAY
            CODE    00CFH     0022H     UNIT         ?PR?INITIAL_UART0?MAIN
            CODE    00F1H     0018H     UNIT         ?PR?MAIN?MAIN
            CODE    0109H     000CH     UNIT         ?C_C51STARTUP
            CODE    0115H     000AH     UNIT         ?PR?_UART0_SEND_BYTE?MAIN



OVERLAY MAP OF MODULE:   MA82G5Dxx (MAIN)


SEGMENT
  +--> CALLED SEGMENT
---------------------
?C_C51STARTUP
  +--> ?PR?MAIN?MAIN

?PR?MAIN?MAIN
  +--> ?PR?INITIAL_UART0?MAIN
  +--> ?PR?_UART0_SEND_BYTE?MAIN



SYMBOL TABLE OF MODULE:  MA82G5Dxx (MAIN)

  VALUE           TYPE          NAME
  ----------------------------------

  -------         MODULE        MAIN
BL51 BANKED LINKER/LOCATER V6.00                                                      07/23/2018  09:53:49  PAGE 2


  C:0000H         SYMBOL        _ICE_DUMMY_
  D:0008H         PUBLIC        flag_Tx0_Busy
  D:0090H         PUBLIC        P1
  D:00A0H         PUBLIC        P2
  D:00C0H         PUBLIC        XICON
  D:00B0H         PUBLIC        P3
  D:00E8H         PUBLIC        P4
  D:00F8H         PUBLIC        P6
  D:00ACH         PUBLIC        SFRPI
  B:00A8H.7       PUBLIC        EA
  D:00A8H         PUBLIC        IE
  D:00B8H         PUBLIC        IP0L
  D:0093H         PUBLIC        T2MOD1
  C:00CFH         PUBLIC        Initial_UART0
  D:00C7H         PUBLIC        CKCON0
  D:00D8H         PUBLIC        CCON
  C:00F1H         PUBLIC        main
  B:00C8H.5       PUBLIC        RCLK_TF2L
  C:0115H         PUBLIC        _UART0_Send_Byte
  D:0089H         PUBLIC        TMOD
  D:0088H         PUBLIC        TCON
  C:0003H         PUBLIC        INT_UART0
  B:00A8H.4       PUBLIC        ES0
  B:0098H.0       PUBLIC        RI0
  B:0098H.1       PUBLIC        TI0
  D:008DH         PUBLIC        TH1
  D:009CH         PUBLIC        S0CFG
  B:0088H.6       PUBLIC        TR1
  D:0099H         PUBLIC        S0BUF
  D:0087H         PUBLIC        PCON0
  D:0098H         PUBLIC        S0CON
  D:00C8H         PUBLIC        T2CON
  B:00C8H.4       PUBLIC        TCLK_TL2IE
  D:00A3H         PUBLIC        AUXR2
  D:00D0H         PUBLIC        PSW
  -------         PROC          INT_UART0
  C:0003H         LINE#         13
  C:0007H         LINE#         16
  C:000AH         LINE#         17
  C:000CH         LINE#         19
  C:0011H         LINE#         20
  C:0011H         LINE#         21
  C:0013H         LINE#         22
  C:0018H         LINE#         23
  C:001BH         LINE#         24
  C:001BH         LINE#         25
  -------         ENDPROC       INT_UART0
  -------         PROC          INITIAL_UART0
  C:00CFH         LINE#         28
  C:00CFH         LINE#         29
  C:00CFH         LINE#         31
  C:00D2H         LINE#         33
  C:00D5H         LINE#         35
  C:00D8H         LINE#         36
  C:00DBH         LINE#         37
  C:00DEH         LINE#         38
  C:00E0H         LINE#         39
BL51 BANKED LINKER/LOCATER V6.00                                                      07/23/2018  09:53:49  PAGE 3


  C:00E2H         LINE#         41
  C:00E5H         LINE#         43
  C:00E8H         LINE#         44
  C:00EBH         LINE#         46
  C:00EEH         LINE#         48
  C:00F0H         LINE#         49
  -------         ENDPROC       INITIAL_UART0
  -------         PROC          _UART0_SEND_BYTE
  D:0007H         SYMBOL        dta
  C:0115H         LINE#         51
  C:0115H         LINE#         52
  C:0115H         LINE#         53
  C:0117H         LINE#         54
  C:011AH         LINE#         55
  C:011EH         LINE#         56
  -------         ENDPROC       _UART0_SEND_BYTE
  -------         PROC          MAIN
  C:00F1H         LINE#         58
  C:00F1H         LINE#         59
  C:00F1H         LINE#         61
  C:00F4H         LINE#         62
  C:00FBH         LINE#         63
  C:00FEH         LINE#         64
  C:0100H         LINE#         65
  C:0102H         LINE#         67
  C:0107H         LINE#         68
  -------         ENDPROC       MAIN
  -------         ENDMOD        MAIN

  -------         MODULE        DELAY_1T
  C:0026H         SEGMENT       CODE_DELAY
  C:00A7H         PUBLIC        DELAY_100US
  C:0086H         PUBLIC        DELAY_10US
  C:0069H         PUBLIC        DELAY_1US
  C:00B2H         PUBLIC        DELAY_200US
  C:0091H         PUBLIC        DELAY_20US
  C:006CH         PUBLIC        DELAY_2US
  C:00C5H         PUBLIC        DELAY_500US
  C:009CH         PUBLIC        DELAY_50US
  C:007BH         PUBLIC        DELAY_5US
  C:0026H         PUBLIC        _DELAY_MS
  D:00E0H         SYMBOL        ACC
  C:0051H         SYMBOL        DELAY_UNIT_1MS
  N:0001H         SYMBOL        FOSC_12MHZ
  N:0000H         SYMBOL        FOSC_24MHZ
  C:0034H         SYMBOL        LSB_LOOP
  C:0041H         SYMBOL        MSB_LOOP0
  C:003EH         SYMBOL        MSB_LOOP1
  C:003AH         SYMBOL        NDLSB
  C:004AH         SYMBOL        NDMSB
  C:0026H         LINE#         29
  C:0028H         LINE#         30
  C:002AH         LINE#         31
  C:002CH         LINE#         33
  C:002EH         LINE#         34
  C:0030H         LINE#         36
  C:0032H         LINE#         37
BL51 BANKED LINKER/LOCATER V6.00                                                      07/23/2018  09:53:49  PAGE 4


  C:0034H         LINE#         39
  C:0037H         LINE#         40
  C:003AH         LINE#         42
  C:003CH         LINE#         43
  C:003EH         LINE#         45
  C:0041H         LINE#         47
  C:0044H         LINE#         48
  C:0047H         LINE#         49
  C:004AH         LINE#         51
  C:004CH         LINE#         52
  C:004EH         LINE#         53
  C:0050H         LINE#         54
  C:0051H         LINE#         57
  C:0054H         LINE#         58
  C:0057H         LINE#         59
  C:005AH         LINE#         60
  C:005DH         LINE#         61
  C:0060H         LINE#         62
  C:0063H         LINE#         63
  C:0066H         LINE#         64
  C:0067H         LINE#         65
  C:0068H         LINE#         66
  C:0069H         LINE#         78
  C:006AH         LINE#         78
  C:006BH         LINE#         79
  C:006CH         LINE#         91
  C:006DH         LINE#         91
  C:006EH         LINE#         91
  C:006FH         LINE#         91
  C:0070H         LINE#         91
  C:0071H         LINE#         91
  C:0072H         LINE#         91
  C:0073H         LINE#         91
  C:0074H         LINE#         91
  C:0075H         LINE#         91
  C:0076H         LINE#         91
  C:0077H         LINE#         91
  C:0078H         LINE#         91
  C:0079H         LINE#         91
  C:007AH         LINE#         92
  C:007BH         LINE#         108
  C:007DH         LINE#         109
  C:0080H         LINE#         110
  C:0083H         LINE#         111
  C:0085H         LINE#         112
  C:0086H         LINE#         127
  C:0088H         LINE#         128
  C:008BH         LINE#         129
  C:008EH         LINE#         130
  C:0090H         LINE#         131
  C:0091H         LINE#         146
  C:0093H         LINE#         147
  C:0096H         LINE#         148
  C:0099H         LINE#         149
  C:009BH         LINE#         150
  C:009CH         LINE#         165
  C:009EH         LINE#         166
BL51 BANKED LINKER/LOCATER V6.00                                                      07/23/2018  09:53:49  PAGE 5


  C:00A1H         LINE#         167
  C:00A4H         LINE#         168
  C:00A6H         LINE#         169
  C:00A7H         LINE#         184
  C:00A9H         LINE#         185
  C:00ACH         LINE#         186
  C:00AFH         LINE#         187
  C:00B1H         LINE#         188
  C:00B2H         LINE#         206
  C:00B4H         LINE#         207
  C:00B7H         LINE#         208
  C:00BAH         LINE#         209
  C:00BDH         LINE#         210
  C:00C0H         LINE#         211
  C:00C2H         LINE#         212
  C:00C3H         LINE#         212
  C:00C4H         LINE#         213
  C:00C5H         LINE#         234
  C:00C8H         LINE#         235
  C:00CBH         LINE#         236
  C:00CEH         LINE#         237
  -------         ENDMOD        DELAY_1T

Program Size: data=10.0 xdata=0 code=284
LINK/LOCATE RUN COMPLETE.  0 WARNING(S),  0 ERROR(S)
